:100000000C94FD070C9435080C9435080C943508B5
:100010000C9435080C9435080C9435080C9435086C
:100020000C9435080C9435080C94BC1D0C94F81CE9
:100030000C94E3230C9435080C9435080C94350883
:100040000C9435080C9435080C9435080C9435083C
:100050000C9435080C94A2230C9435080C943508A4
:100060000C9435080C9435080C9435080C9435081C
:100070000C9435080C9435080C9435080C9435080C
:100080000C9435080C9435080C9435080C943508FC
:100090000C9435080C9435080C9435080C943508EC
:1000A0000C9435080C9435080C9435084410441011
:1000B00076107610EB1007119D129D121211F0119F
:1000C000011201120F1B361BDA1C361BDA1C821BB5
:1000D000A51BDA1C9B1CAA1CA6279427AD271B274F
:1000E00042284228912742284228DC274228F0272C
:1000F00042284228422842284228102842284228E2
:100100000B284228C827422812273C283C283C2894
:100110003C283C283C283C283C283C283E284228B7
:10012000A6278A27422842284228422842284228D5
:1001300042284228422842283E2842284228912725
:1001400042283A283A283A283A283A283A283A2897
:100150003A283A283E2864796E616D6963206D61A2
:1001600063726F207265636F7264696E673A2073A1
:100170007461727465640D0A0064796E616D6963FF
:10018000206D6163726F3A2069676E6F72696E6786
:10019000206D6163726F20706C6179206B657920CE
:1001A0007768696C65207265636F7264696E670D4C
:1001B0000A004B4C3A206B633A2025752C20636F64
:1001C0006C3A2025752C20726F773A2025752C20EB
:1001D000707265737365643A2025750A0044454260
:1001E00055473A2064697361626C65642E0A004465
:1001F000454255473A20656E61626C65642E0A007F
:10020000E600000000004700460000000000E20099
:1002100050004800580057004D004A0000005200AE
:10022000560055005B0061004E004B005E0063000D
:100230004F0054005A006000450049005D00620014
:100240005100530059005F0044004C005C00000066
:10025000380032003300130027002D002F00340037
:10026000000037000F00120026004100400000008F
:10027000000036000E000C0025002E0030003F006C
:10028000110010000D001800240023001C000B00BA
:100290002C00280031000000430042002A003E00EC
:1002A00005001900090015002100220017000A00AE
:1002B000000006000700080020003B003C003D0055
:1002C00000001B0016001A001F003A00E300640043
:1002D00000001D00040014001E0035002B00294200
:1002E0000000E5000000000000000000E100000048
:1002F0000000E400000000000000E000000000003A
:10030000E600000000004700460000000000E20098
:1003100050004800580057004D004A0000005200AD
:10032000560055005B0061004E004B005E0063000C
:100330004F0054005A006000450049005D00620013
:100340005100530059005F0044004C005C00000065
:10035000380032003300130027002D002F00340036
:10036000000037000F00120026004100400000008E
:10037000000036000E000C0025002E0030003F006B
:10038000110010000D001800240023001C000B00B9
:100390002C00280031000000430042002A003E00EB
:1003A00005001900090015002100220017000A00AD
:1003B000000006000700080020003B003C003D0054
:1003C00000001B0016001A001F003A0039006400EC
:1003D00000001D00040014001E0035002B00290041
:1003E0000000E5000000000000000000E100000047
:1003F0000000E400000000000000E0000000000039
:1004000001000000000001000100000000000100E8
:10041000AC00010001000100010001000000A90082
:1004200001000100010001000100010001000100C4
:10043000AB0001000100010001000100010001000A
:10044000AA000100010001000100010001000000FC
:100450000100010001000100010001000100010094
:100460000000010001000100010001000100000086
:100470000000010001000100010001000100010075
:10048000010003530100010001000100010001000F
:10049000AE00010001000000010001000100065D46
:1004A0000100010001000100010001000100010044
:1004B00000000100010001000100085D045D055D10
:1004C00000000100010001000100075D390001008A
:1004D000000001000100010001002B5D010001008E
:1004E000000001000000000000000000010000000A
:1004F00000000100000000000000010000000000FA
:1005000001000000000001000100000000000100E7
:10051000EF00010001000100F300FE000000ED000B
:100520000100010001000100F200FF0001000100D4
:10053000F0000100010001000100FD0001000100C8
:10054000EE000100010001000100F10001000000C7
:100550000100010001000100010001000100010093
:100560000000010001000100010001000100000085
:100570000000010001000100010001000100010074
:100580000100010001000100010001000100010063
:100590000100010001000000010001000100010054
:1005A0000100010001000100010001000100010043
:1005B0000000010001000100010001000100010034
:1005C0000000010001000100010001000100010024
:1005D00000000100010001000100010001000353BF
:1005E0000000010000000000000000000100000009
:1005F00000000100000000000000010000000000F9
:100600004F6E6573686F743A206163746976653AFA
:100610002025640A000A002530325820006B6579D5
:10062000626F6172645F7265706F72743A2000204D
:100630000025303258000D0A5363616E3A200006DF
:1006400031FF0974A1010975150026FF0095207579
:100650000881020976150026FF0095207508910291
:10066000C005010902A10185020901A100050919BE
:100670000129081500250195087501810205010968
:100680003009311581257F950275088106093815D5
:1006900081257F950175088106050C0A38021581B0
:1006A000257F950175088106C0C005010980A1015B
:1006B000850319012AB700150126B70095017510A9
:1006C0008100C0050C0901A101850419012AA002BD
:1006D000150126A002950175108100C005010906CB
:1006E000A101050719E029E7150025019508750105
:1006F00081029501750881010507190029FF150080
:1007000026FF009506750881000508190129059541
:100710000575019102950175039101C05B435D0070
:100720005B445D005B535D005B575D005B525D00A9
:1007300009025B00030100A0FA09040000010301A3
:100740000100092111010001224000070581030871
:10075000000109040100010300000009211101004A
:1007600001227B0007058203200001090402000228
:100770000300000009211101000122220007058366
:1007800003200001070503032000011201000200FD
:10079000000008EDFE8E550100010200012803490A
:1007A0000042004D0020004D006F00640065006CA9
:1007B0000020004D0020003100300031002F0031BA
:1007C0000030003200000016036D00730063006803
:1007D00000770069006E00670065006E000000048D
:1007E00003090464796E616D6963206D6163726FE2
:1007F0003A20736C6F74202564206C656E67746892
:100800003A2025642F25640A0064796E616D69635E
:10081000206D6163726F3A2069676E6F72696E67EF
:100820002061206C656164696E67206B65792D7548
:1008300070206576656E740D0A005B735D000A00BA
:1008400025303862003A200025303258000A722FD5
:10085000632030313233343536370A000A00253010
:100860003258006C65645F7461736B3A2000703AB3
:10087000097072696E742076616C7565730A643AEA
:10088000097365742064656661756C74730A7570AC
:100890003A092B310A646E3A092D310A6C743A090F
:1008A0002B31300A72743A092D31300A4553432FE7
:1008B000713A09717569740A0A7370656564203D3F
:1008C0002064656C7461202A206D61785F737065A7
:1008D0006564202A2028726570656174202F207459
:1008E000696D655F746F5F6D6178290A77686572FD
:1008F000652064656C74613A20637572736F723D34
:1009000025642C20776865656C3D25640A53656510
:1009100020687474703A2F2F656E2E77696B69703A
:10092000656469612E6F72672F77696B692F4D6FF0
:100930007573655F6B6579730A004D3E20004D2528
:10094000753A25733E20003F0A003D2025750A00B8
:100950003F0A0064656661756C74730A0025750A48
:10096000003F0A000A092D2056616C756573202D21
:100970000A00710A000A092D204D6F7573656B65B9
:1009800079202D0A004C25640A0064796E616D6936
:1009900063206D6163726F3A20736C6F74202564FD
:1009A00020706C61796261636B0A0064796E616DBD
:1009B0006963206D6163726F3A20736C6F742025D8
:1009C000642073617665642C206C656E6774683A88
:1009D0002025640A0064796E616D6963206D61632E
:1009E000726F3A207472696D6D696E672061207450
:1009F0007261696C696E67206B65792D646F776EC3
:100A0000206576656E740D0A00290A002575002F91
:100A1000002575005D280025640020002564002065
:100A20000025640020002564007C00253032580039
:100A30006D6F7573656B6579205B62746E7C782071
:100A400079207620685D287265702F61636C293A81
:100A5000205B006B65796D61705F636F6E666967BF
:100A60002E7261773A20253032580A2E73776170E2
:100A70005F636F6E74726F6C5F636170736C6F63D2
:100A80006B3A2025750A2E636170736C6F636B5F20
:100A9000746F5F636F6E74726F6C3A2025750A2EE7
:100AA000737761705F6C63746C5F6C6775693A2013
:100AB00025750A2E737761705F7263746C5F72675D
:100AC00075693A2025750A2E737761705F6C616CC9
:100AD000745F6C6775693A2025750A2E73776170AB
:100AE0005F72616C745F726775693A2025750A2EB2
:100AF0006E6F5F6775693A2025750A2E737761708E
:100B00005F67726176655F6573633A2025750A2EAB
:100B1000737761705F6261636B736C6173685F624E
:100B200061636B73706163653A2025750A2E6E6B85
:100B3000726F3A2025750A0064656275675F636F9E
:100B40006E6669672E7261773A20253032580A2E18
:100B5000656E61626C653A2025750A2E6D6174724E
:100B600069783A2025750A2E6B6579626F61726427
:100B70003A2025750A2E6D6F7573653A2025750A22
:100B8000006565636F6E6669673A0A6465666175DC
:100B90006C745F6C617965723A2025750A000A09E8
:100BA0002D204D61676963202D0A443A094465622E
:100BB0007567204D65737361676520546F67676C57
:100BC000650A583A094D6174726978204465627506
:100BD00067204D6F646520546F67676C65202D201A
:100BE00053686F77206B65797072657373657320D6
:100BF000696E206D617472697820677269640A4B4E
:100C00003A094B6579626F61726420446562756769
:100C100020546F67676C65202D2053686F77206BB9
:100C200065797072657373207265706F72740A4DA6
:100C30003A094465627567204D6F75736520546F7E
:100C400067676C650A563A0956657273696F6E0A72
:100C5000533A095374617475730A433A09416374D2
:100C6000697661746520436F6E736F6C65204D6F9C
:100C700064650A46312D4631303A09537769746309
:100C80006820746F204C6179657220302D392028DE
:100C9000463130203D204C30290A302D393A095355
:100CA000776974636820746F204C617965722030B5
:100CB0002D390A47524156453A095377697463689A
:100CC00020746F204C6179657220302028616C742B
:100CD00065726E617465290A423A094A756D702021
:100CE000746F20426F6F746C6F616465720A455354
:100CF000433A094A756D7020746F20426F6F746CAF
:100D00006F616465722028616C7465726E617465D0
:100D1000290A453A095072696E7420454550524F70
:100D20004D2053657474696E67730A425350414392
:100D3000453A09436C65617220454550524F4D0A52
:100D40005A3A09536C656570204C454420546573CC
:100D5000740A000A092D20436F6E736F6C65202D95
:100D60000A4553432F713A09717569740A6D3A093E
:100D70006D6F7573656B65790A000A092D205665DC
:100D80007273696F6E202D0A5649443A20307846B6
:100D9000454544286D73636877696E67656E2920E1
:100DA0005049443A203078353538452849424D205D
:100DB0004D6F64656C204D203130312F3130322938
:100DC000205645523A203078303030310A42554969
:100DD0004C443A2020284665622032382032303296
:100DE00032290A4F5054494F4E533A204C554641F0
:100DF000204D4F5553454B45592045585452414B72
:100E0000455920434F4E534F4C4520434F4D4D4184
:100E10004E44204C544F20343039360A4743433A2D
:100E200020352E342E30204156522D4C4942433A23
:100E300020322E302E30204156525F415243483AE4
:100E400020617672350A000A092D20537461747589
:100E500073202D0A686F73745F6B6579626F6172BE
:100E6000645F6C65647328293A20253032580A6B18
:100E70006579626F6172645F70726F746F636F6CBB
:100E80003A20253032580A6B6579626F6172645F6F
:100E900069646C653A20253032580A74696D657250
:100EA0005F72656164333228293A202530386C58E6
:100EB0000A003F000A6D6F7573653A206F66660A17
:100EC000000A6D6F7573653A206F6E0A000A6B65D4
:100ED00079626F6172643A206F66660A000A6B6518
:100EE00079626F6172643A206F6E0A000A6D6174F4
:100EF0007269783A206F66660A000A6D61747269D9
:100F0000783A206F6E0A000A64656275673A206F4E
:100F100066660A000A64656275673A206F6E0A00A9
:100F20000A0A4A756D70696E6720746F20626F6F70
:100F3000746C6F616465722E2E2E2000433E20007B
:100F4000436C656172696E6720454550524F4D0A8A
:100F500000536C656570204C454420546573740AD9
:100F600000313A0964656C6179282A31306D732942
:100F70003A2025750A323A09696E74657276616C99
:100F8000286D73293A2025750A333A096D61785F17
:100F900073706565643A2025750A343A0974696D81
:100FA000655F746F5F6D61783A2025750A353A097F
:100FB000776865656C5F6D61785F73706565643ACD
:100FC0002025750A363A09776865656C5F74696D26
:100FD000655F746F5F6D61783A2025750A003F0088
:100FE000433E20004C4544205570646174653A20AE
:100FF0002564202564202564000011241FBECFEF46
:10100000DAE0DEBFCDBF04B603FE18C08091200633
:1010100090912106A0912206B09123068730904B33
:10102000A740B04B59F4109220061092210610925E
:10103000220610922306E0E0F8E3099511E0A0E013
:10104000B1E0E6EFFCE502C005900D92AC3DB107C2
:10105000D9F726E0ACEDB1E001C01D92A032B20795
:10106000E1F70E94ED1E0C94792E0C940000FF9382
:10107000EF93E091DC01F091DD01309709F00995E3
:10108000EF91FF910895FC018591803011F0EFDF21
:10109000FBCF0895FF27E0E230E247FF0CC0419507
:1010A00097FF09C0EDE26095709580959095611D60
:1010B000711D811D911D27FF02C0219530E350E273
:1010C000AA27660F771F881F991FAA1FA41710F061
:1010D000A41B63955A95A9F7AA3008F0A95FA05DF3
:1010E000AF93F395611571058105910541F7ED32D7
:1010F00011F4EF93F395F21718F43F93F395FBCFA8
:101100008F91B5DFFA95E1F70895E991F99185910D
:10111000803021F0853219F0AADFF9CF089520E060
:10112000E89455915532C1F3503311F468945591B8
:101130005A3348F4505390F3220F022E220F220FFD
:10114000200D250FF4CF0EF42195899199915336F6
:1011500019F3533729F1533559F1BC0188279927E1
:10116000E8945C3621F489919991689455915436AC
:1011700039F446EF7EF077FF0DC08FEF9FEF0AC086
:1011800055374AE039F0583540E121F0523642E017
:1011900009F00895FF93EF937DDFEF91FF91B7CFB3
:1011A000FF93EF93FC0181918030B9F360DFFBCFB7
:1011B000FF93EF9368DFF1CFDF93CF93CDB7DEB727
:1011C0002596A3DFCF91DF9108952F923F924F9202
:1011D0005F926F927F928F929F92AF92BF92CF92C7
:1011E000DF92EF92FF920F931F93CF93DF93CDB7D0
:1011F000DEB72F970FB6F894DEBF0FBECDBFFC0150
:10120000F080118183819481892B39F01F3F39F45B
:1012100091E00FEFF01203C003C091E001C090E035
:1012200090FF02C00C9408133F0185E0DE01169682
:1012300001900D928A95E1F7D30112962C918E813F
:101240009F81222349F00E94602A082F682F8E81F7
:101250009F810E94E52A03C00E94B92A082FE12F2E
:10126000F0E0B0E10B9FE00DF11D112463E0EE0F03
:10127000FF1F6A95E1F7EF0DF11DEE0FFF1FE05024
:10128000FE4FA591B491BF87AE874D01CD0181502E
:1012900095458F3F910520F4FD01B5E5FB2702C080
:1012A000EE85FF85D3011296BC91BC87BB2309F460
:1012B000BEC2EF3FF10579F070F0EB32FD4519F059
:1012C0001092FE0179C49091FE0181E089278093FC
:1012D000FE010C94DE128091FE01882309F4E8C01F
:1012E0001092FE01E03CF10540F4E038F10508F011
:1012F00073C0E034F105D0F505C0EF3FF10509F00A
:1013000008F4A0C021E030E040E050E060E070E090
:1013100080E090E00E2F0E94362EA091DE012A2B55
:10132000A091DF013A2BA091E0014A2BA091E101AD
:101330005A2BA091E2016A2BA091E3017A2BA09194
:10134000E4018A2BA091E5019A2B2093DE013093D2
:10135000DF014093E0015093E1016093E20170935B
:10136000E3018093E4019093E50128C421E030E09B
:1013700040E050E060E070E080E090E08F010054D9
:1013800011090E94362EA091E6012A2BA091E701B7
:101390003A2BA091E8014A2BA091E9015A2BA09188
:1013A000EA016A2BA091EB017A2BA091EC018A2B28
:1013B000A091ED019A2B2093E6013093E701409331
:1013C000E8015093E9016093EA017093EB01809387
:1013D000EC019093ED01F2C321E030E040E050E0F9
:1013E00060E070E080E090E08F01005811090E94F9
:1013F000362EA091EE012A2BA091EF013A2BA0915D
:10140000F0014A2BA091F1015A2BA091F2016A2B15
:10141000A091F3017A2BA091F4018A2BA091F50100
:101420009A2B2093EE013093EF014093F0015093FB
:10143000F1016093F2017093F3018093F4019093B2
:10144000F501BCC321E030E040E050E060E070E036
:1014500080E090E08F01005C11090E94362EA0917F
:10146000F6012A2BA091F7013A2BA091F8014A2B03
:10147000A091F9015A2BA091FA016A2BA091FB01CE
:101480007A2BA091FC018A2BA091FD019A2B20932D
:10149000F6013093F7014093F8015093F9016093FE
:1014A000FA017093FB018093FC019093FD0186C3C8
:1014B000E034F105D0F45090DE01A090DF01B0904F
:1014C000E001E090E101F090E2011091E3018090F1
:1014D000E4019090E50121E030E040E050E060E080
:1014E00070E080E090E00E2F5DC0E038F105E8F498
:1014F0005090E601A090E701B090E801E090E9018A
:10150000F090EA011091EB018090EC019090ED01D8
:1015100021E030E040E050E060E070E080E090E00A
:101520006F01A0E4CA1AD1083CC0E03CF105E8F420
:101530005090EE01A090EF01B090F001E090F10129
:10154000F090F2011091F3018090F4019090F50178
:1015500021E030E040E050E060E070E080E090E0CA
:101560006F01B0E8CB1AD1081CC05090F601A090D2
:10157000F701B090F801E090F901F090FA011091B4
:10158000FB018090FC019090FD0121E030E040E003
:1015900050E060E070E080E090E06F0100ECC01A85
:1015A000D1080C2D0E94362E5222232E2A20342EB2
:1015B0003B20452E4E20F622E72EE122A82FA8211F
:1015C000B92FB92121E030E040E050E060E070E068
:1015D00080E090E0E034F10580F08F01E038F10523
:1015E00018F4005411090AC0E03CF10518F4005841
:1015F000110904C0005C110901C00E2F0E94362E93
:1016000059016A014B018C01252D322D432D542D9A
:101610006F2D7E2DCD0174010E944F2E09F0CCC29A
:10162000E03CF10548F4E038F10508F084C0E0340E
:10163000F10508F042C005C0EF3FF10509F008F4DC
:10164000B8C021E030E040E050E060E070E080E0D1
:1016500090E00E2F0E94362E2095309540955095A3
:101660006095709580959095E091DE012E23E09134
:10167000DF013E23E091E0014E23E091E1015E2392
:10168000E091E2016E23E091E3017E23E091E40129
:101690008E23E091E5019E232093DE013093DF014C
:1016A0004093E0015093E1016093E2017093E30104
:1016B0008093E4019093E50181C78F0100541109E3
:1016C00021E030E040E050E060E070E080E090E059
:1016D0000E94362E209530954095509560957095D6
:1016E00080959095E091E6012E23E091E7013E235D
:1016F000E091E8014E23E091E9015E23E091EA01E7
:101700006E23E091EB017E23E091EC018E23E091CA
:10171000ED019E232093E6013093E7014093E80119
:101720005093E9016093EA017093EB018093EC011F
:101730009093ED0143C78F010058110921E030E07B
:1017400040E050E060E070E080E090E00E94362EE3
:101750002095309540955095609570958095909521
:10176000E091EE012E23E091EF013E23E091F001A4
:101770004E23E091F1015E23E091F2016E23E091AE
:10178000F3017E23E091F4018E23E091F5019E2385
:101790002093EE013093EF014093F0015093F1015B
:1017A0006093F2017093F3018093F4019093F5013B
:1017B00005C78F01005C110921E030E040E050E0F6
:1017C00060E070E080E090E00E94362E2095309539
:1017D000409550956095709580959095E091F601B3
:1017E0002E23E091F7013E23E091F8014E23E09192
:1017F000F9015E23E091FA016E23E091FB017E2363
:10180000E091FC018E23E091FD019E232093F601DF
:101810003093F7014093F8015093F9016093FA0176
:101820007093FB018093FC019093FD01C7C6EF3FCD
:10183000F10511F008F0C4C0E034F105D0F4509087
:10184000DE01A090DF01B090E001E090E101F090B6
:10185000E2011091E301B091E401A091E50121E0E2
:1018600030E040E050E060E070E080E090E00E2F7B
:101870005DC0E038F105E8F45090E601A090E70182
:10188000B090E801E090E901F090EA011091EB01DD
:10189000B091EC01A091ED0121E030E040E050E09A
:1018A00060E070E080E090E06F0100E4C01AD108D1
:1018B0003CC0E03CF105E8F45090EE01A090EF014F
:1018C000B090F001E090F101F090F2011091F3017D
:1018D000B091F401A091F50121E030E040E050E04A
:1018E00060E070E080E090E06F0100E8C01AD1088D
:1018F0001CC05090F601A090F701B090F801E09064
:10190000F901F090FA011091FB01B091FC01A09156
:10191000FD0121E030E040E050E060E070E080E078
:1019200090E06F0100ECC01AD1080C2D0E94362EF9
:101930005222332E3A20242E2B20E522F622472E47
:101940004122B8239A239B87E034F105C0F08F0130
:10195000E038F10518F40054110908C0E03CF10525
:1019600018F40058110902C0005C110921E030E0B0
:1019700040E050E060E070E080E090E009C021E0ED
:1019800030E040E050E060E070E080E090E00E2F5A
:101990000E94362E59016A01F62FE72F8C01A1E033
:1019A000252D332D422D5E2D6F2D742D8B2F9B8574
:1019B000EF2EFE2E0E944F2E09F4A0E08A2F01C0C8
:1019C00081E080FFFBC58091FF0481115AC0AC8586
:1019D000A111F6C0B5E08B16BDE59B0681F130F490
:1019E000F4E08F16FDE59F06A1F0EAC007E080163F
:1019F0000DE59006E1F118E081161DE5910609F06C
:101A0000DFC060910001709101014FEF89EF94E018
:101A100035C08091720580FF04C086E591E00E9488
:101A200043080E94AA2D0E948F2B0E94602B8FEFEB
:101A300091E0909371058093700581E015C08091CD
:101A4000720580FF04C086E591E00E9443080E9471
:101A5000AA2D0E948F2B0E94602B89EF94E0909317
:101A600071058093700582E08093FF04A7C56091A3
:101A700002017091030141E08FEF91E00E94512536
:101A80009DC524E082162DE59206C8F137E0831645
:101A90003DE5930630F099E089169DE5990640F101
:101AA0002EC091E0A6E08A16ADE59A0609F490E012
:101AB000BC85B91709F482C5813061F08230A9F480
:101AC000609170057091710520E031E04FEF89EF72
:101AD00094E009C0609170057091710522E031E0D9
:101AE00041E08FEF91E00E94E9241092FF0466C567
:101AF0008091720580FF62C589E791E05AC081300C
:101B000061F0823009F05CC06091020170910301C4
:101B100093014FEF89EF94E008C06091000170914C
:101B20000101930141E08FEF91E00E947D1948C0CF
:101B3000D30112968C91882309F409C21092B20540
:101B4000B4E08B16BDE59B0608F0A4C0EBEF8E1643
:101B5000ECE59E0608F0A9C0C40182509C4544975C
:101B600008F4A3C016E181161CE5910609F4DDC155
:101B70008FED88168CE5980609F419C208F001C2A9
:101B80008114ACE59A0609F40CC2B1E08B16BCE5F1
:101B90009B0609F01AC280917205982F909591705A
:101BA00090FB80F980937205992309F4FDC18FEEB3
:101BB00091E00E94430802C5EE85FF854F0103CFE7
:101BC0008091720580FF17C0F30182811F928F936D
:101BD00081811F928F9380811F928F939F928F920A
:101BE00082EB91E09F938F930E94DC080FB6F894EC
:101BF000DEBF0FBECDBF14EF81161CE5910679F153
:101C0000B0F439ED83163CE5930619F18AED881698
:101C10008CE59806B1F198ED89169CE5990609F0D6
:101C200087CF06E221EE41EE68ED7CE52FC0A6EFFE
:101C30008A16ACE59A06F9F0C0F0E7EF8E16ECE5EF
:101C40009E0609F075CF07E225EE46EE67EF7CE5CC
:101C50001DC007E225EE45EE69ED7CE517C006E202
:101C600021EE40EE64EF7CE511C007E225EE44EE84
:101C700065EF7CE50BC006E221EE42EE66EF7CE507
:101C800005C008E221E045EE6AED7CE5C3010E9453
:101C90005E2494C4F2E68F16FDE59F0631F006EA55
:101CA00080160DE5900609F05DCF0E94FE1490931A
:101CB00084058093830511E181161CE5910609F4E2
:101CC000DAC008F04BC039E083163CE5930609F40E
:101CD000AEC028F595E089169CE5990609F497C0F1
:101CE00090F4B3E08B16BCE59B0609F489C008F0BC
:101CF0008BC0F2E08F16FCE59F0609F006C18091CB
:101D00008305816000C107E080160CE5900609F4A8
:101D100086C008F088C0809183058061F4C02DE002
:101D200082162CE5920609F494C060F48BE08816C4
:101D30008CE5980609F485C008F087C0809183057A
:101D400088607BC0AFE08A16ACE59A0609F48BC0C8
:101D500008F08DC080918305877FD5C0EEEF8E1689
:101D6000ECE59E0609F47BC028F505E180160CE53C
:101D7000900609F48EC070F423E182162CE59206D9
:101D800009F47DC008F09DC00E948F2B80918305CF
:101D90008F77B9C08CEF88168CE59806E1F108F0D2
:101DA0005BC0ABEF8A16ACE59A0609F0AEC0809135
:101DB000840545C0B2E08B16BDE59B0609F48DC0D5
:101DC00058F48114FDE59F0609F45EC008F06DC06B
:101DD00080918405826033C012E681161DE591066C
:101DE00009F481C026EA82162DE5920609F485C021
:101DF00033E083163DE5930609F087C060E06EC0CE
:101E00008091830582607FC08091830516C0809198
:101E10008305886078C08091840582604FC080917E
:101E20008305806270C08091830580646CC00E94CD
:101E30008F2B80918305806866C0846064C0816058
:101E40003DC0809183058E7F5EC0809183058D7F2C
:101E50005AC08091830516C08091840518C0809176
:101E600084058D7F2BC0809183058F7E4CC080912F
:101E700083058F7D48C0809183058F7B44C080910E
:101E80008305877F8B7F3FC0809184058D7F8E7F08
:101E900015C08091830582FB222720F991E09227CB
:101EA00090FB82F990FB83F92EC080918405982FD6
:101EB000909591708E7F892B90FB81F9809384059A
:101EC00024C00E948F2B8091830587FB222720F955
:101ED00091E0922790FB87F916C061E08EE090E0D8
:101EE0000E94DC2D12C08091830584FB222720F9FB
:101EF00091E0922790FB84F906C080918305982F8A
:101F0000909590FB80F980938305609183051091F3
:101F1000840584E090E00E94DC2D612F82E290E055
:101F20000E94DC2D0E948F2B49C380914B058A7A39
:101F300091E009F490E090930005882311F065E3A7
:101F400001C069E281E095E00E940C2417C0B6E16F
:101F50008B16BCE59B06C9F580910005882309F422
:101F600055C385E3E1E0F5E027E035E09281891390
:101F700001C0128231962E173F07C1F70E948715C4
:101F80001DC3ECE58E16EDE59E06E1F0FDE58F162E
:101F90009F0681F00BE580160DE59006B1F481E017
:101FA00012C00E947B2D0AC38DED91E002CE0E94EB
:101FB0000F1504C38091840582FB882780F991E086
:101FC000892701C080E00E941E16D30112968C91D1
:101FD00012970C9111961C91882349F0C8010E9418
:101FE000602AF82E682FC8010E94E52A04C0C801A3
:101FF0000E94B92AF82EE12FF0E0B0E1FB9EE00D3F
:10200000F11D112433E0EE0FFF1F3A95E1F7E00FC9
:10201000F11DEE0FFF1FE050FE4F859194910E943D
:1020200064138C01B82EF301F280C580C2945FE086
:10203000C522809141058770B9F0FF20A9F0812F5A
:10204000807F803421F080E2800F883068F08091BA
:10205000840582FD09C082E00E940116809141053D
:102060008770EE24E3948111E12CD12ED2942FE0DD
:10207000D2228D2D90E08C30910508F05EC2FC01DB
:10208000EA5AFF4F0C94302E812F807F1F708823D7
:1020900011F01295107FFF20B9F0112309F43AC214
:1020A00080E2800F883010F0B11006C080914B059F
:1020B000182B10934B0505C080914A05182B1093DF
:1020C0004A050E94871526C2802F0E94AB2B112340
:1020D00009F433C2005E083078F1BB2069F1109535
:1020E00080914A05182310934A0529C0812F807FCB
:1020F0001F70803211F01295107FBB2021F0F1E0AB
:10210000BF16D9F149C08091840582FF1BC0FF2012
:1021100069F0112339F080914B05182B10934B0572
:102120000E94871580E00E94E32B07C280E00E9496
:10213000AB2B112309F401C2812F0E9480150E944C
:102140008715FBC1FF2081F080914C05CC2051F018
:1021500001E0C01207C0182B181709F4EEC1109344
:102160004C05EBC1812B10C0CC2021F021E0C21620
:1021700009F4E3C10E947A152AC0FF2041F035E03E
:102180003C1508F4DAC1812F0E94A12BD6C184E04E
:102190008C1508F4D2C11BC0FF2061F0CC2099F34C
:1021A000D30115968C91159780FFB4C18F70159649
:1021B0008C93E9CFCC2059F0093309F0BBC1BFEFB4
:1021C000E7EEF3E0B150E040F040E1F7B1C1812F1C
:1021D0000E949A2BB2C1812F86958695837019F043
:1021E000813059F0AAC1FF2019F0C801937002C0D4
:1021F00080E090E00E943C24A8C1FF2019F0C801B3
:10220000937002C080E090E00E9426249EC1802F3F
:10221000FF2019F00E943E2902C00E944F280E9410
:10222000992993C1812F837009F069C0F11089C188
:10223000902F929596959770990F990F802F8F7088
:10224000882E912CA12CB12C092E04C0880C991C2D
:10225000AA1CBB1C0A94D2F704FF12C04FE050E046
:1022600060E070E004C0440F551F661F771F9A9509
:10227000D2F7DB01CA0180959095A095B09503C077
:1022800080E090E0DC0116951695412F43704230B6
:1022900019F1C8F400914D0510914E0520914F059C
:1022A00030915005413059F088299929AA29BB2934
:1022B000BC01CD0160237123822393230AC0802AAD
:1022C000912AA22AB32ABC01CD01682979298A2939
:1022D0009B290E94652B35C188299929AA29BB29E8
:1022E00000914D0510914E0520914F0530915005FC
:1022F000BC01CD016027712782279327EACFFF20F9
:1023000019F0812F817001C08695882309F419C1C5
:10231000902F929596959770990F990F802F8F70A7
:10232000882E912CA12CB12C092E04C0880C991C4C
:10233000AA1CBB1C0A94D2F704FF12C04FE050E065
:1023400060E070E004C0440F551F661F771F9A9528
:10235000D2F7DB01CA0180959095A095B09503C096
:1023600080E090E0DC0116951695412F43704230D5
:10237000D9F068F50091AB051091AC052091AD0541
:102380003091AE05413059F088299929AA29BB29F5
:10239000BC01CD0160237123822393231EC0802AB8
:1023A000912AA22AB32A13C088299929AA29BB29CC
:1023B0000091AB051091AC052091AD053091AE05B3
:1023C000BC01CD01602771278227932706C0BC017D
:1023D000CD01682979298A299B290E94102BB1C037
:1023E0001F70FF2039F0812F0E943F2B802F0E9409
:1023F000A12BA7C0802F0E949A2B812F0E941A2BFD
:10240000A0C0802F22EFB21609F443C02B1538F07C
:1024100030EFB31659F091EFB916B1F176C0A3EFD2
:10242000BA16F1F1B4EFBB1659F16FC0FF2019F1E4
:10243000E4E0EC1508F481C01F7181E090E0A0E0B9
:10244000B0E0AC01BD0104C0440F551F661F771FEB
:102450001A95D2F78091AB059091AC05A091AD058E
:10246000B091AE058A019B01082719272A273B272F
:10247000C901B80125C025E02C1508F45EC0DCCFE9
:102480008091840582FF22C0FF2029F0812F8F7167
:102490002FC0FF20D9F3812F8F710E941A2B4DC0BE
:1024A000FF2089F01F7181E090E0A0E0B0E0BC0166
:1024B000CD0104C0660F771F881F991F1A95D2F7A8
:1024C0000E94102B3AC00E94602B37C0FF2099F069
:1024D0001F71812F0E943F2B8091840582FD07C0D0
:1024E00038E0139FC0011124836080934105812F40
:1024F0000E943F2B22C081E00E94011681E08C15D2
:10250000E0F482E00E94011618C0FF2029F0CC20E0
:1025100009F4BCCF802F07CECC2009F4BCCF89337F
:1025200049F49FEFA7EEB3E09150A040B040E1F72F
:1025300000C00000802F0E94AB2B88EF8D0D8430EF
:1025400020F40E9452240E942F2DEE20A9F08091A9
:10255000410580FD11C0F301128285958595859511
:102560000E943F2BC3010E94E5088091410585959B
:10257000859585950E941A2B85E0F301DE01119661
:1025800001900D928A95E1F789819A810E94B92A7A
:10259000EA81F0E000E1809FE00DF11D112483E06D
:1025A000EE0FFF1F8A95E1F78981E80FF11DEE0F0D
:1025B000FF1FE050FE4F859194912AC08091410504
:1025C000877031F1D30112968C91882309F18091A3
:1025D000840582FD1DC082E02F960FB6F894DEBF01
:1025E0000FBECDBFDF91CF911F910F91FF90EF9064
:1025F000DF90CF90BF90AF909F908F907F906F9023
:102600005F904F903F902F900C94011689E2AACCD6
:102610002F960FB6F894DEBF0FBECDBFDF91CF91DE
:102620001F910F91FF90EF90DF90CF90BF90AF90F0
:102630009F908F907F906F905F904F903F902F90E2
:1026400008959091830592FF0DC0282F287128309E
:1026500019F4877F846006C0282F2471243011F478
:102660008B7F886093FF0DC0282F2871283119F4C3
:10267000877E846106C0282F2471243111F48B7E5B
:1026800088612091840520FF0DC0382F38713830C3
:1026900019F4877F816006C0382F3171313011F411
:1026A0008E7F886021FF0DC0282F2871283119F4F2
:1026B000877E816106C0282F2171213111F48E7E21
:1026C000886194FD877E0895CF93DF9382389105CA
:1026D00069F1B0F48133910509F46FC048F489328F
:1026E000910509F465C08A32910509F46BC08AC06E
:1026F0008533910509F457C089339105B9F082C03B
:10270000833E910571F138F4803E9105B1F0823E2F
:10271000910511F177C0863E9105B9F1873E91058B
:10272000C9F1843E910509F06DC024C02091830554
:1027300020FD53C021FD51C065C08091830580FDFF
:1027400046C08091840580FF48C08091830584FD48
:1027500050C183EE90E04FC18091830582FF3AC063
:10276000F4CF8091830582FD35C08091840580FD82
:1027700034C0EBCF8091840581FF35C08091830503
:1027800084FD37C187EE90E036C18091830583FFD9
:1027900027C0F4CF8091830583FD22C080918405FA
:1027A00081FD21C0EBCF8091830585FD1FC021C035
:1027B0008091830585FD1DC019C08091830586FD2C
:1027C0001BC01DC08091830586FD19C015C089E31B
:1027D00090E011C182EE90E00EC180EE90E00BC15E
:1027E00086EE90E008C184EE90E005C189E290E0B9
:1027F00002C185E390E0FFC08AE290E0FCC081E383
:1028000090E0F9C0811531E5930708F069C08115A2
:1028100040E59407F0F09C0174E0369527957A9591
:10282000E1F7922F9370482F437021E030E002C00F
:10283000220F331F4A95E2F73C68392B982F9F707F
:102840009695969540E2949FC0011124822B932B7C
:10285000D2C0883E910568F5803E910508F0CBC056
:10286000883A9105B8F4853A910548F0855AE82FE1
:10287000F0E0E95EFE4F808190E09064BCC0813062
:10288000910509F4B3C008F4B4C08430910508F48C
:10289000B0C0B1C08F3B910508F0ABC0885AE82F9B
:1028A000F0E0EE0FFF1FE65EFE4F808191819464A1
:1028B000A2C0811520E2920758F4811531E09307F8
:1028C00008F099C08D3E910508F493C0906593C0BF
:1028D000811540E4940708F48CC09F70906A8BC007
:1028E000811525E5920708F042C0811534E593076C
:1028F00028F0982F8827846F906A7DC0811543E562
:102900009407B0F09C012370332741E050E002C0EF
:10291000440F551F2A95E2F7282F2695269580E229
:10292000289F90011124CA01822B932B9A6863C0BF
:10293000811522E5920728F4982F8827816F906AE5
:102940005AC09C012370332741E050E002C0440F7D
:10295000551F2A95E2F7282F2695269580E2289F75
:1029600090011124CA01822B932B9C6844C0EC0176
:10297000811539E59307A8F48115984528F09C2F17
:102980008827806F906A37C0C11586E5D80788F51B
:102990008C2F0E9421138F7190E0982F88279062CE
:1029A0002AC081152AE5920790F48C2F8F700E941F
:1029B000211394E0D695C7959A95E1F7CF70D0E0B2
:1029C000DC2FCC27D0699E01282BC90114C090565A
:1029D0008115904270F48D2F8F710E942113282F42
:1029E0002F71CE0199279062922B05C081E090E073
:1029F00002C080E090E0DF91CF910895CF9384E012
:102A000090E00E94CE2DC82F82E290E00E94CE2D51
:102A10002C2F30E0A901582BCA01CF91089569EEFF
:102A20007EEF80E090E00E94FA2D60E082E090E08E
:102A30000E94DC2D60E083E090E00E94DC2D10928B
:102A40004D0510924E0510924F051092500560E012
:102A500084E090E00E94DC2D60E082E290E00E9441
:102A6000DC2D60E085E090E00E94DC2D60E086E0F7
:102A700090E00E94DC2D6FEF87E090E00E94DC2D5B
:102A800040E050E0BA0188E090E00E94EE2D60E066
:102A90008DE090E00E94DC2D40E050E0BA0188E13A
:102AA00090E00E94EE2D60E087E190E00E94DC2D36
:102AB00040E050E0BA018CE190E00E94EE2D60E031
:102AC00070E080E290E00E94FA2D40E050E0BA0110
:102AD00088E190E00E94EE2D40E050E0BA018FE0E6
:102AE00090E00E94EE2D40E050E0BA0183E190E0DA
:102AF0000C94EE2D80914C05811110924C05089597
:102B0000809590914B05892380934B050895EF9212
:102B1000FF920F931F93CF9390914B0580914A059D
:102B2000982B9093010580914C05882389F0892B7F
:102B300080930105E3E0F5E097E080E0915029F013
:102B400021912223D9F38F5FF9CF81110E947A1549
:102B500048E050E062E475E081E095E00E946C2E70
:102B6000892B09F448C088E0E1E0F5E0A2E4B5E093
:102B700001900D928A95E1F7E091B505F091B605C7
:102B80003097C9F10280F381E02D81E095E009954D
:102B90008091720582FF2FC080FF04C08DE196E016
:102BA0000E94430801E015E0C8E087E1E82E86E0D6
:102BB000F82E8091720580FF0CC0F80180811F9271
:102BC0008F93FF92EF920E94DC080F900F900F906E
:102BD0000F90C1500F5F1F4FC111EBCF8091720555
:102BE00080FF09C085E196E0CF911F910F91FF9082
:102BF000EF900C944308CF911F910F91FF90EF90AD
:102C00000895209141058095822380934105982F56
:102C1000977099F430E0482F082E000C550B2417BC
:102C2000350759F09091840592FD07C085958595EB
:102C300085950E941A2B109241050895CF93DF933A
:102C4000C0918405C2FB992790F9981719F1D82FE4
:102C500080FBC2F9C09384056091830584E090E015
:102C60000E94DC2D6C2F82E290E00E94DC2D82E03D
:102C70000E9401168091720580FF0CC01F92DF93A5
:102C800080E096E09F938F930E94DC080F900F9056
:102C90000F900F90DF91CF91089580914005909112
:102CA0000F05891719F08F5F8770FBCF08950F9379
:102CB0001F93CF93DF9380910E0582958F7009F05B
:102CC0005DC080910B05882309F458C080914005B0
:102CD00010910F056091090570910A05C0910C05CE
:102CE000D0910D0591E06F3F09F090E0292F06E0AB
:102CF000811709F443C0209721F07F3F21F030E095
:102D000003C031E001C0322F90E030FD34C0089F95
:102D1000F001099FF00D1124DF01A05FBA4F119659
:102D20003C911197371327C03C91361324C012965B
:102D30003C91129731111FC013964D915C911497DD
:102D40004C1B5D0B483C5105B0F480910E058F7013
:102D5000806180930E05EB5EFA4F80818F708061F9
:102D6000808389E095E00E94E508DF91CF911F9173
:102D70000F910C944D1601968770BACFDF91CF91C9
:102D80001F910F910895CF93DF93D82FC92F0E94E1
:102D9000602AEC2FF0E090E1899FE00DF11D1124F5
:102DA00083E0EE0FFF1F8A95E1F7ED0FF11DEE0FA7
:102DB000FF1FE050FE4F859194910E946413DF91B4
:102DC000CF9108959F92AF92BF92CF92DF92EF92F0
:102DD000FF920F931F93CF93DF93CDB7DEB7619729
:102DE0000FB6F894DEBF0FBECDBF8C0185E0F801B1
:102DF000DE011D9601900D928A95E1F7F801E280BF
:102E00009091090560910A0540910C0550910D05BE
:102E10004115510531F06F3F31F481E09F3F19F4C6
:102E200003C081E001C080E0F82FF1709F2E80FD8B
:102E30001AC1F80130812181C380D48089E0A82E95
:102E400085E0B82EF0900B05F601E41BF50BFF2092
:102E500009F4C6C080910E05E83CF10508F091C068
:102E6000482F407F09F050C0621311C093130FC068
:102E7000FE2CE1100CC08F70806180930E05C5019F
:102E80000E94E50880910E05F801858329C1CD28AF
:102E900031F02F3F31F481E03F3F19F403C081E06E
:102EA00001C080E080FD03C081E08E2502C080E08B
:102EB00090E0F82FF170FF2E80FF1CC0809140053C
:102EC00040910F0556E0841709F4E8C090E0589F40
:102ED000F001599FF00D1124E05FFA4F6181261334
:102EE00006C06081631303C06281E61203C00196CD
:102EF0008770E9CFFE2CEE2009F4F2C080910E0518
:102F0000816080930E0549C0621306C0931304C00C
:102F1000E11002C0F80186C0C8010E946F2B88230F
:102F200051F1EE2041F120910E05822F82958F7094
:102F300090E0029774F08091090590910A059887B6
:102F40008F831986DB86CA862C87CE0107960E945E
:102F5000E50886E0F801A9E0B5E001900D928A95B8
:102F6000E1F70E9457160AC06217C9F0C8010E9413
:102F70006F2B81111EC0C8010E94E508FF24F39445
:102F8000AFC0482F407F81F789E095E00E94E508B7
:102F900086E0F50111928A95E9F7F12CA1C093130F
:102FA000E5CFE110E3CFF8018583C8010E94E50871
:102FB00054C0EE2001F320910E05822F82958F7070
:102FC00090E0029734F28091090590910A059A8366
:102FD00089831B82DD82CC822E83CE010196B7CFFE
:102FE000E83CF105D0F5FE2CEE2029F2621327C053
:102FF000931325C020910E0520FD18C0822F8295C5
:103000008F70482F50E04115510581F0F80125835C
:103010004F30510541F08F5F982F9295907F822F0E
:103020008F70892B8583C8010E94E50886E0F8012E
:10303000A9E0B5E001900D928A95E1F751C0C80171
:103040000E946F2B811185CF80910E058160809346
:103050000E05C8010E94E50843C086E0F501119203
:103060008A95E9F73DC0EE2009F485CFC8010E949A
:103070006F2BF82E882309F47ECF86E0F801A9E0B3
:10308000B5E001900D928A95E1F780910905909144
:103090000A050E94C3160E94571622C03D872E873C
:1030A0008D859E850E94C316292F22952F70223070
:1030B00028F49F7039F0811105C00BC0243028F42A
:1030C0009F7049F4805E883020F0C8010E94E508B6
:1030D0009F2CF92C05C0F8019581907F99F7F9CFC5
:1030E0008F2D61960FB6F894DEBF0FBECDBFDF9176
:1030F000CF911F910F91FF90EF90DF90CF90BF90F5
:10310000AF909F9008953F924F925F926F927F92FF
:103110008F929F92AF92BF92CF92DF92EF92FF92E7
:103120000F931F93CF93DF938091720580FF04C0AC
:1031300086E396E00E94430827E7C22E21E0D22EC4
:10314000C0E0D0E0312CEE24E394F12C41E3842E56
:1031500046E0942E1C2FD6018C91E82FE295EF705B
:10316000F0E021A18F70A70102C0440F551F8A957E
:10317000E2F7CA01922F982B91A392A180958923FF
:1031800082A350EA5A95F1F72898289A0E94B62D02
:10319000782E612C0E94B62D5C01A628B72880915C
:1031A000720580FF0DC0C501809590959F938F9308
:1031B0009F928F920E94DC080F900F900F900F90BB
:1031C0008091720580FF04C08FE296E00E94430860
:1031D000C70101C0880F1A95EAF7282F809503E7E9
:1031E00015E0A8E4B1E093E8492E95E0592EF801E6
:1031F00030E060814D915D914A215B21962F452BF6
:1032000011F4922B01C09823691711F0908331E0DB
:10321000319695E0E338F90761F7D6018D916D019C
:10322000E82FE295EF70F0E021A18F70A70102C0B6
:10323000440F551F8A95E2F7CA01942F9095922367
:1032400091A392A1892B82A3332A2196C830D1055C
:1032500009F080CF8091AF058823D1F0809152058D
:10326000909153050E94C8238739910588F0C09139
:10327000510581E0C827C09351050E94D723909340
:10328000530580935205CC2311F02D9A01C02D983F
:10329000332049F081E0809356050E94D723909314
:1032A00055058093540580915605882399F08091A7
:1032B0005405909155050E94C823059758F0E5E8FC
:1032C000F5E0D8018D918D0181934A165B06C9F70F
:1032D00010925605832DDF91CF911F910F91FF9092
:1032E000EF90DF90CF90BF90AF909F908F907F90A6
:1032F0006F905F904F903F900895CF93DF93EC01D4
:10330000F9018281A0917005B091710581110DC004
:10331000AC17BD0751F48091720580FF6CC089E045
:1033200098E0DF91CF910C94430826E04202C0015F
:1033300011249D01281B390B6217730779F036E0C1
:1033400001900D923A95E1F7209170053091710549
:10335000820F931F90937105809370058091720581
:1033600080FF49C0E42F042E000CFF0B6C1B7D0B6B
:1033700075956795ABEABAEA6A9FC0016B9F900D9D
:103380007A9F900D11248E9F90018F9F300D9E9FEC
:10339000300D11242F5F3F4F809170059091710582
:1033A0008C1B9D0B959587958A9FE0018B9FD00D77
:1033B0009A9FD00D1124CE9FB001CF9F700DDE9F3C
:1033C000700D1124141614F082E001C081E03F93C7
:1033D0002F937F936F931F928F9383EE97E09F932A
:1033E0008F930E94DC088DB79EB708960FB6F894AD
:1033F0009EBF0FBE8DBFDF91CF910895EF92FF92D8
:103400000F931F93CF93DF937C018B010E94BD220A
:10341000811119C0E70101151105A1F08091E800A3
:1034200085FD0AC08091E8008E778093E8000E94B5
:10343000BD22882381F307C089918093F100015058
:103440001109E9CF80E0DF91CF911F910F91FF909B
:10345000EF9008951F93CF93DF93CDB7DEB7AA9770
:103460000FB6F894DEBF0FBECDBFE8E6F5E0809161
:10347000F100819345E0E037F407C9F780916905D1
:10348000833009F461C030F4813071F0823009F486
:103490009BC0B2C08A3009F487C08B3009F46CC07D
:1034A000893009F0A9C020C080916805813A09F0EF
:1034B000A3C08091E800877F8093E80080916C052D
:1034C00090916D05892B21F468E08CE595E003C0AF
:1034D00060E080E090E070E00E9444238091E8008A
:1034E0008B778093E80088C080916805813209F06D
:1034F00083C080916C0590916D05029708F07CC0A7
:103500008091E800877F8093E8008091E80082FD49
:1035100005C0809166058111F8CF6EC02091F3003F
:103520008091F20090E0922B029731F48091F100AB
:10353000813011F0863021F48091F10080935B0599
:103540008091E8008B7754C080916805813A09F03A
:1035500053C080916C0590916D05892B09F04CC08A
:103560008091E800877F8093E8008091E80080FFE9
:10357000FCCF8091040137C0809168058132E1F56C
:1035800080916C0590916D05892BB1F58091E800D3
:10359000877F8093E8000E94F02280916A058093E3
:1035A00004010E948F2B28C080916805813221F58B
:1035B0008091E800877F8093E8000E94F02280914C
:1035C0006B0580935A0518C080916805813AA1F473
:1035D0008091E800877F8093E8008091E80080FF79
:1035E000FCCF80915A058093F1008091E8008E779E
:1035F0008093E8000E94F0228091E80083FFDAC106
:103600008091680590916905492F50E04A30510535
:1036100008F0D0C1FA01EE59FF4F0C94302E8038DB
:1036200021F0823809F0C6C108C0809164059091EC
:103630006505992389F082600FC080916C058F70B9
:10364000873008F0B7C18093E9008091EB0085FBDB
:10365000882780F91092E9009091E800977F909375
:10366000E8008093F1001092F10070C1282F2D7FA7
:1036700009F0A0C1882319F0823061F09BC18091CC
:103680006A05813009F096C1933009F080E080939B
:1036900065052EC080916A0581112AC080916C0554
:1036A0008F702FEF280F263008F084C18093E90037
:1036B0002091EB0020FF1CC0933021F48091EB009F
:1036C000806214C09091EB0090619093EB0021E038
:1036D00030E0A90102C0440F551F8A95E2F74093DC
:1036E000EA001092EA008091EB0088608093EB0082
:1036F0001092E9008091E800877F8093E8000E94A3
:10370000F02258C1811156C110916A051F7780912E
:10371000E3008078812B8093E3008091E800877F2D
:103720008093E8000E94F0228091E80080FFFCCFA7
:103730008091E30080688093E300111102C082E071
:1037400001C083E08093660535C18058823008F05F
:1037500031C120916A0530916B052C3D53E035074E
:1037600079F583E08A838AE289834FB7F894DE0192
:10377000139620E03EE051E2E32FF0E05093570033
:10378000E49120FF03C0E295EF703F5FEF708E2F52
:1037900090E0EA3010F0C79601C0C0968D939D93DB
:1037A0002F5F243149F74FBF8091E800877F8093D6
:1037B000E8006AE270E0CE0101960E944423B5C0A1
:1037C00080916C0590916D05432F5527433051052D
:1037D000A9F068F44130510509F4FBC042305105AD
:1037E00009F0E8C08BE590E0E0E3F7E04BC0413240
:1037F000510529F14232510589F1DCC0C9019927EF
:1038000081309105A1F058F0029709F0D3C0EDE99D
:10381000F7E0E4918E2F90E0EDE9F7E030C0EFEDB6
:10382000F7E0E4918E2F90E0EFEDF7E028C0E7ECB1
:10383000F7E0E4918E2F90E0E7ECF7E020C08330D2
:10384000910508F0B7C0880F991FFC01EF58FE4F93
:103850000190F081E02D89E090E014C08330910563
:1038600008F0A8C0FC01EE0FFF1FE559FE4F0190C4
:10387000F081E02DDC01A859BE4F8C9190E00097BB
:1038800009F498C02091E800277F2093E800209158
:103890006E0530916F058217930708F49C0140E094
:1038A0002115310589F180916605882309F43DC011
:1038B0008530D9F18091E80083FD37C08091E80020
:1038C00082FD2FC08091E80080FFEACF4091F30095
:1038D0008091F20090E0942B2115310559F0883049
:1038E000910540F444914093F10031962150310903
:1038F0000196F2CF41E0089709F040E08091E8009E
:103900008E778093E800CCCF4111CDCF0AC0809153
:103910006605882351F0853041F08091E80083FDF1
:1039200004C08091E80082FFF2CF8091E8008B779D
:103930008093E8003FC08038E9F58091E800877FF8
:103940008093E800809167058093F1008091E80002
:103950008E77D3CE81112EC080916A0590916B0530
:10396000992702973CF58091E800877F8093E800D3
:1039700010916A05109367050E94F022111106C08C
:103980008091E30087FD02C081E001C084E0809364
:10399000660542E061EC81E00E940F2342E261ECA7
:1039A00082E00E940F2342E261EC83E00E940F2339
:1039B000809166058091E80083FF10C08091E80047
:1039C000877F8093E8008091EB0080628093EB001A
:1039D00005C082E190E0EBE8F7E054CFAA960FB67D
:1039E000F894DEBF0FBECDBFDF91CF911F91089538
:1039F0001F920F920FB60F9211242F933F934F9364
:103A00005F936F937F938F939F93AF93BF93CF9366
:103A1000DF93EF93FF93C091E900CF708091EC00AA
:103A2000D82FD17080FDD0E81092E9008091F0008D
:103A3000877F8093F00078940E942A1A1092E90000
:103A40008091F00088608093F000CD2BCF70C09300
:103A5000E900FF91EF91DF91CF91BF91AF919F91DD
:103A60008F917F916F915F914F913F912F910F9027
:103A70000FBE0F901F901895E8EDF0E080818E7FCB
:103A800080831092E2001092DA001092E100A0EE22
:103A9000B0E08C9181608C9380818F77808319BC9A
:103AA000A7EDB0E08C918E7F8C9380818F7E808398
:103AB000109259050895CF92DF92EF92FF920F93E3
:103AC0001F93CF93DF93C8EDD0E088818F7E8883EA
:103AD000E7EDF0E080818160808384E082BF81E057
:103AE0008093590588818E7F888302EE10E0F8016B
:103AF00010821092DA0081EEC82ED12CF6011082CD
:103B000088818F77888388818068888388818F7D8A
:103B1000888319BC1092660510926705109265059E
:103B20001092640590EEE92EF12CF70180818B7FD5
:103B3000808388818160888342E060E080E00E9429
:103B40000F23F60180818E7F8083F8018081816060
:103B50008083808188608083F70180818E7F80836D
:103B6000888180618883DF91CF911F910F91FF90B1
:103B7000EF90DF90CF9008951F920F920FB60F92A3
:103B800011242F933F934F935F936F937F938F9362
:103B90009F93AF93BF93EF93FF938091E10082FFD8
:103BA00049C08091E20082FF45C08091E1008B7F97
:103BB0008093E100209158052F5F822F62E30E94DD
:103BC000102E992319F02093580534C010925805EF
:103BD00080915705882371F180916605843041F505
:103BE0008091E9008F702091EC00922F917020FD60
:103BF00090E8892B93E09093E9009091EB0090FF7F
:103C000014C09091EE0097FF10C09091E80095FFCE
:103C100003C01092F100F9CF9091E80090FF05C029
:103C20009091E8009E779093E8008F708093E90070
:103C3000109257058091DA0080FF32C08091D80041
:103C400080FF2EC08091DA008E7F8093DA00809111
:103C5000D90080FF1CC080E189BD82E189BD09B423
:103C600000FEFDCF81E0809366058CE197E00E9425
:103C7000430880915905811113C00E943C1D0E9488
:103C80005B1D8091E20084608093E20009C019BC52
:103C90001092660580E297E00E9443081092590551
:103CA0008091E10080FF1CC08091E20080FF18C07D
:103CB0008091E2008E7F8093E2008091E20080613B
:103CC0008093E2008091D80080628093D80019BC74
:103CD00085E08093660584E297E00E944308769829
:103CE0008091E10084FF39C08091E20084FF35C0FB
:103CF00080E189BD82E189BD09B400FEFDCF8091DC
:103D0000D8008F7D8093D8008091E1008F7E8093D2
:103D1000E1008091E2008F7E8093E2008091E200DA
:103D200081608093E20080916705882311F084E030
:103D300007C08091E30087FD02C081E001C083E0FD
:103D40008093660588E297E00E94430880916605AB
:103D5000769A0E9452240E942F2D8091E10083FFC9
:103D60002BC08091E20083FF27C08091E100877F14
:103D70008093E10082E08093660510926705809150
:103D8000E1008E7F8093E1008091E2008E7F80933E
:103D9000E2008091E20080618093E20042E060E016
:103DA00080E00E940F238091F00088608093F000F3
:103DB0008CE297E00E944308FF91EF91BF91AF9191
:103DC0009F918F917F916F915F914F913F912F9133
:103DD0000F900FBE0F901F901895CF93DF93CDB724
:103DE000DEB763970FB6F894DEBF0FBECDBF84B7C2
:103DF000877F84BF0FB6F894A89580916000886192
:103E000080936000109260000FBE90E080E80FB6D3
:103E1000F89480936100909361000FBE85B780682D
:103E200085BF85B7806885BF8CED91E29093DD01F9
:103E30008093DC01269A509A259A2E9858982D98AE
:103E40006E9A769A0FEF10E722E001501040204062
:103E5000E1F700C00000209A219A229A29980E9436
:103E60003C1D0E945B1D8091E20084608093E20013
:103E70007894809166058823A1F01091E9001F7065
:103E80009091EC00892F817090FD80E8182B1092A2
:103E9000E9008091E80083FD0E942A1A1F701093A8
:103EA000E90082E084BD93E095BD9AEF97BD8093D1
:103EB0006E00A7E7B1E04FE751E061E070E08D915F
:103EC000E82FE295EF70F0E021A18F708B0102C026
:103ED000000F111F8A95E2F7C801902F9095922349
:103EE00091A392A1892B82A34A175B0741F71DBCBE
:103EF00088E58CBDE3E7F5E083E895E0A5E8B5E06B
:103F000011921D928E179F07D9F780E090E00E94D2
:103F1000D62D893E9E4F11F00E940F1582E090E051
:103F20000E94CE2D809372050E94FE14909384050A
:103F30008093830583E090E00E94CE2D682F70E08F
:103F400080E090E00E94652B85E091E09093B605BB
:103F50008093B50545E9242E45E0342E58E4452EDE
:103F600058E0552E60E4662E68E0762E8091660556
:103F7000853009F04DC08AE398E00E94430830E4A0
:103F8000F32E00E112E180916605853009F03AC018
:103F900080916605843031F180E00E942F2D1092CF
:103FA000B90528E130E00FB6F894A8952093600099
:103FB0000FBEF092600083B7817F846083BF83B7B8
:103FC000816083BF7894889583B78E7F83BF0FB657
:103FD000F894A895809160008861809360001092A9
:103FE00060000FBE80916505882309F4CCCF0E9444
:103FF0008318E5E8F5E081918111BFC12E163F06D7
:10400000D1F7C1CF0E948F2B0E9452240E942F2DE6
:104010000E948318882359F08FB7F8944091BA050D
:104020005091BB056091BC057091BD058FBF95E9AE
:10403000C92E95E0D92E25E8A22E25E0B22E00E06B
:1040400010E00B8BF50121915F012A8BF601819124
:104050006F012827298B211116C00F5F1F4F0031D8
:10406000110579F78FEF8C878D871E860E94D723E5
:104070008160782F988B8F874C855D856E858889C8
:104080000E94872C5BC08091720581FD04C080E096
:10409000FF24F39435C08DE498E00E94430885E83E
:1040A000882E85E0982EE12CF12CFF92EF925F9202
:1040B0004F920E94DC0885E498E00E944308F401D6
:1040C00081914F010E94692D1F928F937F926F9271
:1040D0000E94DC088EE398E00E944308FFEFEF1A8D
:1040E000FF0A0FB6F894DEBF0FBECDBF30E1E31676
:1040F000F104D9F6CCCF8F5FFF0C883009F4ADCF37
:1041000099899F21C1F38F834B8948879A899F2181
:1041100081E009F480E089870E94D7238160782FAD
:104120009B878A874F81588569858B850E94872C5C
:10413000F801EB56FA4F8081F826F08286E0E9EC30
:10414000F5E0DE01119601900D928A95E1F7E0907D
:10415000CB05F090CC050091CD051091CE051092C5
:10416000CB051092CC051092CD051092CE05E11032
:1041700003C0FF2009F45DC08091C7059091C80578
:104180000E94C823AC019091C405992339F0209175
:10419000150130E02417350758F04BC02091160167
:1041A0008AE0289F900111242417350718F041C098
:1041B0009F3F19F09F5F9093C405EE2061F00E942D
:1041C000FF281E1414F09FEF01C091E0899F802DFD
:1041D00011248093CB05FF2061F00E94FF281F145B
:1041E00014F09FEF01C091E0899F802D11248093EE
:1041F000CC053091CB053323E1F02091CC0522236F
:10420000C1F045EB3403C0011124992319F09093B8
:10421000CB0503C081E08093CB0535EB2303C001C0
:104220001124992319F09093CC0503C081E0809369
:10423000CC05011103C0112309F451C08091C505BB
:104240009091C6050E94C8239C019091C2059923B4
:1042500009F4A9C02135310508F441C09F3F19F088
:104260009F5F9093C205002361F00E94C62810163C
:1042700014F09FEF01C091E0899F802D112480935D
:10428000CD05112361F00E94C628111614F09FEF8E
:1042900001C091E0899F802D11248093CE0530913B
:1042A000CD053323E1F02091CE052223C1F045EB6B
:1042B0003403C0011124992319F09093CD0503C054
:1042C00081E08093CD0535EB2303C00111249923B0
:1042D00019F09093CE0503C081E08093CE058091C4
:1042E000CB0581110BC08091CC05811107C0809155
:1042F000CD05811103C08091CE0581110E949929BD
:10430000EB82FC820D831E8386E0FE013196A9ECD0
:10431000B5E001900D928A95E1F70E945224182F82
:104320008091A505181709F421CE1093A505809159
:10433000720582FF1EC080FF04C083E698E00E94E1
:1043400043088091720580FF0CC01F921F938EE579
:1043500098E09F938F930E94DC080F900F900F902E
:104360000F908091720580FF04C08CE598E00E9458
:104370004308812F0E942F2DF9CD09BD19BD09B425
:1043800000FEFDCF8091D8008F7D8093D800809172
:10439000E00082608093E0008091E00081FDFCCF2E
:1043A0000E948F2BF0CD2B30310508F059CF97CFDD
:1043B000089580915B0508959FB7F8941092570572
:1043C0009FBF90916605943009F057C09091E90025
:1043D0009F703091EC00232F217030FD20E8922B4C
:1043E00023E02093E9002091EB0020FF43C02091BF
:1043F000EE0027FF3FC02091C105222321F020912C
:10440000E80025FF37C01092C10526E03091E80092
:1044100035FD15C030916605343061F53091EB0003
:1044200035FD28C0215021F481E08093C10522C0D0
:10443000EFE9FFE03197F1F700C00000E7CF80938C
:10444000F1008091E80085FD0AC08091E80080FFBE
:10445000FCCF8091E8008E778093E80006C08FB78C
:10446000F89421E0209357058FBF9F709093E90047
:1044700080E008959F709093E9008FEF08958093F6
:10448000BE057093C0056093BF05809166058430BA
:1044900001F582E08093E9008FEF9091E800815070
:1044A00095FD06C095ED9A95F1F700008111F5CFC5
:1044B0008091E80085FF0DC040E050E063E070E0CF
:1044C0008EEB95E00E94FE198091E8008E77809334
:1044D000E8000895BC0184E00C943F22BC0183E015
:1044E0000C943F2222E02093E9002FEF3091E80066
:1044F000215035FD06C035ED3A95F1F70000211148
:10450000F5CF2091E80025FF0BC040E050E066E0C9
:1045100070E00E94FE198091E8008E778093E80099
:104520000895CF93DF9321E02093E9002FEF30919E
:10453000E800215035FD06C035ED3A95F1F7000051
:104540002111F5CF2091E80025FF14C0EC0140E0D7
:1045500050E068E070E00E94FE198091E8008E77DC
:104560008093E80088E0FE01ACE5B5E001900D9293
:104570008A95E1F7DF91CF9108952091E400309181
:10458000E50095E64091EC00842F817040FF23C048
:104590008091E80080FD1DC080916605882399F018
:1045A000853099F08091EB0085FD11C04091E400C9
:1045B0005091E5002417350729F3915011F09A0125
:1045C000E1CF84E0089582E0089583E0089581E0DA
:1045D000089580E008954091E80042FFDDCF0895FE
:1045E0008091680587FF11C08091E80082FD05C0B9
:1045F000809166058111F8CF11C08091E8008B771A
:104600000BC080916605882349F08091E80080FF07
:10461000F8CF8091E8008E778093E8000895982F76
:10462000973068F59093E900981739F07091EC0095
:104630002091ED005091F00003C0242F762F50E020
:1046400021FD02C09F5FECCF3091EB003E7F3093A5
:10465000EB003091ED003D7F3093ED003091EB00A9
:1046600031603093EB007093EC002093ED00509399
:10467000F0002091EE0027FDE5CF80E008958F70D7
:104680008093E90081E0089520916E0530916F05D7
:104690002617370748F06115710539F42091E800B5
:1046A0002E772093E80001C0B901FC0120E06115DC
:1046B000710579F1809166058823F1F18530F1F17A
:1046C0008091E80083FD3CC08091E80082FD2EC00F
:1046D0008091E80080FFEBCF2091F3008091F20001
:1046E00090E0922B6115710551F08830910538F4F6
:1046F00021912093F100615071090196F3CF21E0DF
:10470000089709F020E08091E8008E778093E80018
:10471000CECF2111CFCF0AC080916605882361F0EA
:10472000853061F08091E80083FD0AC08091E80047
:1047300082FFF2CF80E0089582E0089583E008953B
:1047400081E0089578941F920F920FB60F92112472
:104750008F939F93AF93BF938091BA059091BB05C0
:10476000A091BC05B091BD050196A11DB11D80931E
:10477000BA059093BB05A093BC05B093BD05BF914E
:10478000AF919F918F910F900FBE0F901F90189532
:104790009C014FB7F8948091BA059091BB05A09108
:1047A000BC05B091BD054FBF821B930B08952FB779
:1047B000F8948091BA059091BB05A091BC05B09189
:1047C000BD052FBF08951F920F920FB60F921124AF
:1047D0008F939F93AF93BF938091B905811113C0BD
:1047E0008091BA059091BB05A091BC05B091BD0523
:1047F0004196A11DB11D8093BA059093BB05A0936E
:10480000BC05B093BD05BF91AF919F918F910F9063
:104810000FBE0F901F9018959C01FC0132969FEFE0
:1048200080E04191461789F09F3F19F4411101C082
:10483000982F8F5F8630A9F79F3F39F0F901E90F74
:10484000F11D97FDFA956283089508952091B705AB
:104850003091B8052817390771F09093B805809307
:10486000B705E091B505F091B605309721F00084C9
:10487000F185E02D099408952091B3053091B40598
:104880002817390771F09093B4058093B305E09130
:10489000B505F091B605309721F00680F781E02D3F
:1048A00009940895E091B505F091B605309721F08F
:1048B0000190F081E02D099480E00895EF92FF923D
:1048C0000F93CF93DF93C42FD22FFC0182818823D3
:1048D000D1F04093B2050E94D7239093B105809305
:1048E000B00580E28C0F883008F06DC0C77081E0A1
:1048F00001C0880FCA95EAF7DF91CF910F91FF9021
:10490000EF900C94A12B8091B20548134BC080917D
:10491000B0059091B1050E94C823883C910508F02C
:1049200041C0CD17C9F080E28C0F883040F4C770C9
:1049300081E001C0880FCA95EAF70E949A2B80E2B5
:104940008D0F883048F481E09D2F977001C0880F4B
:104950009A95EAF70E94A12B093319F0E12CF12C6A
:1049600003C080E5E82EF12C802F0E94E32BE11498
:10497000F10451F08FE99FE00197F1F700C00000CA
:1049800091E0E91AF108F3CF802F0E94AB2B80E26F
:104990008D0F8830C0F4D77081E001C0880FDA95A0
:1049A000EAF70AC080E28C0F883068F4C77081E0B3
:1049B00001C0880FCA95EAF7DF91CF910F91FF9060
:1049C000EF900C949A2BDF91CF910F91FF90EF9085
:1049D00008958F929F92AF92BF92CF92DF92EF9203
:1049E000FF921F93CF93DF936C01EB01142F79019A
:1049F0008091AF05882319F081508093AF058AEF2D
:104A000018024001112480917205CC15DD0519F4BE
:104A100080FD10C037C05E01A80CB91CF501928161
:104A20009923B1F380FF04C085ED99E00E9443080B
:104A3000E501E9CFCE018C199D09959587952BEA63
:104A40003AEA829FA001839F500D929F500D11243E
:104A500014039001159F300D1124111614F082E0FB
:104A600001C081E03F932F931F928F938BEA99E0CF
:104A70009F938F930E94DC080F900F900F900F90E0
:104A80000F900F90F701D183C083DF91CF911F91D9
:104A9000FF90EF90DF90CF90BF90AF909F908F905E
:104AA00008958F929F92AF92BF92EF92FF920F93D1
:104AB0001F93CF93DF93EC017B01042F809172054C
:104AC00080FF11C0141614F082E001C081E01F9233
:104AD0008F938AE899E09F938F930E94DC080F9050
:104AE0000F900F900F908090AB059090AC05A09028
:104AF000AD05B090AE050E948F2B0E94602B86E022
:104B0000080280011124CE15DF0531F0CE010E948C
:104B1000E508C00FD11FF7CF0E948F2BC501B4014C
:104B2000DF91CF911F910F91FF90EF90BF90AF90C9
:104B30009F908F900C94102BCF93C82F1F928F9320
:104B400085E899E09F938F930E94DC0881E090E0D4
:104B5000A0E0B0E0BC01CD0104C0660F771F881F44
:104B6000991FCA95D2F70E94652B0F900F900F9056
:104B70000F90CF910C948F2B883220F58E3108F056
:104B800068C08B3091F1C0F4873009F0BEC081E07D
:104B90008093160184E1809315018AE080931401CB
:104BA0008EE18093130188E08093120188E2809364
:104BB000110183E599E0C6C0833109F443C0843113
:104BC00069F1A3C08F3409F49EC028F4893231F111
:104BD000883359F09AC0813531F008F4D4C0823559
:104BE00009F4A7C092C08FEFA5C085E799E00E94A5
:104BF00043080E94D9261F9281E08F931F9288E07C
:104C00008F938EE698E09F938F930E94DC080F901D
:104C10000F900F900F900F900F9096C082E799E041
:104C20000E9443088091AA05882309F4AAC0109223
:104C3000AA051092A9051092A8051092A705109236
:104C4000A605B1C084E699E00E9443080E94D926D7
:104C50007BC08D518093AA05833031F170F481308F
:104C6000D1F0823009F03FC085E191E09093A90531
:104C70008093A8058CE891E01FC0853059F108F1B8
:104C8000863089F581E191E09093A9058093A8058C
:104C900087EC91E011C086E191E09093A9058093A3
:104CA000A80583E891E008C084E191E09093A9050C
:104CB0008093A80588E991E09093A7058093A605C5
:104CC00018C083E191E09093A9058093A80585EA37
:104CD00091E0F2CF82E191E09093A9058093A8053D
:104CE00084EB91E0E9CF1092AA0581E699E00E9459
:104CF00043088091AA05882309F455C01F928F9319
:104D00008DE599E00DC08AE015C080E599E01AC0F4
:104D100097FF47C0108280811F928F938AE499E0A9
:104D20009F938F930E94DC080F900F900F900F902D
:104D30000BC081E0E091A805F091A905309729F515
:104D400087E499E00E9443082091AA05222359F1A3
:104D50008091A6059091A705009711F48FE791E047
:104D60009F938F931F922F938EE399E09F938F933E
:104D70000E94DC080F900F900F900F900F900F90F3
:104D800016C080E0089586EFD5CF2081082E000C54
:104D9000990B820F911D8F3F910509F00CF4B8CF4C
:104DA0008FEF8083B8CF8AE399E00E94430881E0C7
:104DB0000895809111011F928F93809112011F928B
:104DC0008F93809113011F928F93809114011F92F2
:104DD0008F93809115011F928F93809116011F92DE
:104DE0008F9381E69FE09F938F930E94DC088DB79D
:104DF0009EB70E960FB6F8949EBF0FBE8DBF089556
:104E0000CF92DF92EF92FF92CF93DF93482F50E043
:104E1000FA013597EF33F10508F034C1E459FF4F3B
:104E20000C94302E81E59FE00E9443080E9452249A
:104E30000E942F2D6DC083E090E00E94CE2D1F9226
:104E40008F9381E89BE09F938F930E94DC0882E020
:104E500090E00E94CE2D83FB992790F91F929F939B
:104E600082FB992790F91F929F9381FB992790F9D4
:104E70001F929F93982F91701F929F931F928F93D1
:104E800088E39BE09F938F930E94DC080E94FE14AE
:104E900087FB222720F91F922F9386FB222720F9D8
:104EA0001F922F9385FB222720F91F922F9384FBBB
:104EB000222720F91F922F9383FB222720F91F928C
:104EC0002F9382FB222720F91F922F9391FB2227F9
:104ED00020F91F922F93292F21701F922F9381FB6E
:104EE000222720F91F922F93282F21701F922F9392
:104EF0009F938F9383E59AE09F938F930E94DC08A2
:104F00008DB79EB788960FB6F8949EBF0FBE8DBF23
:104F1000C1E0BDC080E49FE00E9443080E940F15DD
:104F2000F7CF8EE99BE079C080917205817F8E7FFB
:104F30008093720583E59DE00E9443088CE39FE027
:104F40000E94430881E08093CF05E2CF80E29FE09A
:104F50000E9443080E947B2DDBCF80917205C82FF1
:104F6000C095C170C0FB80F980937205CC2329F0F5
:104F700084E19FE00E9443088AC087E09FE00E948E
:104F8000430880917205897F877F80937205C0CF27
:104F90009091720591FBCC27C0F981E0C827892F39
:104FA000C0FB81F980937205CC2319F08AEF9EE053
:104FB00027C08CEE9EE031C09091720592FBCC2709
:104FC000C0F981E0C827892FC0FB82F98093720560
:104FD000CC2319F08DED9EE013C08DEC9EE01DC03A
:104FE0009091720593FBCC27C0F981E0C827892FE7
:104FF000C0FB83F980937205CC2351F081EC9EE0D5
:105000000E944308809172058160809372053FC0C1
:1050100084EB9EE002C08AE79DE00E94430878CFBF
:105020008FB7F894C090BA05D090BB05E090BC054E
:10503000F090BD058FBFD0915A05C09104010E9428
:105040005224FF92EF92DF92CF921F92DF931F9232
:10505000CF931F928F9387E49EE09F938F930E943C
:10506000DC088DB79EB70C960FB6F8949EBF0FBEA6
:105070008DBF4ECF895303C08D5101C080E00E9487
:105080009C2546CF82EB9EE00E944308C0E08C2F17
:10509000DF91CF91FF90EF90DF90CF9008958D3EFC
:1050A00039F49091CC0597FF35C01092CC0559C0CA
:1050B0008E3E29F49091CC051916BCF32BC090912B
:1050C000CB058F3E29F497FF25C01092CB0549C030
:1050D000803F19F41916CCF31DC09091CD05893F7E
:1050E00029F41916BCF41092CD053BC08A3F19F47F
:1050F00097FF10C0F8CF8B3F39F49091CE0597FF02
:1051000009C01092CE052DC08C3F21F49091CE05A0
:105110001916BCF39FE0980F983080F421E030E03E
:10512000A90102C0440F551F9A95E2F7CA01809564
:105130009091CA0589238093CA0513C08D3F21F43D
:105140008091C3058E7F0BC08E3F21F48091C305F3
:105150008D7F05C08F3F29F48091C3058B7F80939D
:10516000C3058091CB05811106C08091CC058111CA
:1051700002C01092C4058091CD05811106C08091B6
:10518000CE05811102C01092C20508958091C30519
:1051900080FF08C06091120170E075956795759564
:1051A000679521C081FF06C06091120170E075957E
:1051B000679519C082FF04C06091120170E010C0B1
:1051C0009091C205992399F0609111019617A0F76B
:1051D00080911201899FC001112470E00E941C2E51
:1051E0006038710540F46115710519F406C061E07D
:1051F00070E0862F08958FE7089581E008958091EB
:10520000C30580FF06C06091140170E0660F771F30
:1052100026C081FF04C06091140184E005C082FFB4
:1052200007C06091140188E0689FB001112417C085
:105230009091C4059923D1F060911301961788F7D6
:105240002091140188E0289F90011124929FA001D1
:10525000939F500D112470E0CA010E941C2E6038EB
:10526000710540F46115710519F406C068E070E03D
:10527000862F08958FE7089581E008958D3E21F4EB
:105280000E94FF28819504C08E3E29F40E94FF28C9
:105290008093CC0508958F3E21F40E94FF288195CC
:1052A00004C0803F29F40E94FF288093CB05089515
:1052B000893F19F40E94C62805C08A3F31F40E9434
:1052C000C62881958093CD0508958B3F21F40E94D7
:1052D000C628819504C08C3F29F40E94C62880937B
:1052E000CE0508959FE0980F983078F421E030E0E3
:1052F000A90102C0440F551F9A95E2F7CA01909187
:10530000CA05892B8093CA0508958D3F21F48091A9
:10531000C30581600BC08E3F21F48091C30582607C
:1053200005C08F3F29F48091C30584608093C30535
:1053300008958091720583FF7EC080E39AE00E9409
:1053400043088091CA051F928F938BE29AE09F9346
:105350008F930E94DC0889E29AE00E9443088091C2
:10536000CB05282F082E000C330B3F938F9386E23A
:105370009AE09F938F930E94DC0884E29AE00E9457
:1053800043088091CC05282F082E000C330B3F9347
:105390008F9381E29AE09F938F930E94DC088FE1C4
:1053A0009AE00E9443088091CD05282F082E000C1A
:1053B000330B3F938F938CE19AE09F938F930E94DE
:1053C000DC088AE19AE00E9443088091CE05282FEC
:1053D000082E000C330B3F938F9387E19AE09F9345
:1053E0008F930E94DC0884E19AE00E944308809138
:1053F000C4051F928F9381E19AE09F938F930E943F
:10540000DC088FE09AE00E9443088091C3051F9258
:105410008F938CE09AE09F938F930E94DC0889E041
:105420009AE00E9443088DB79EB74C960FB6F89449
:105430009EBF0FBE8DBF0E94D7232091CB052111A7
:1054400004C02091CC05222321F09093C8058093BD
:10545000C7052091CD05211104C02091CE0522233E
:1054600021F09093C6058093C505E091B505F091B4
:10547000B605309749F082E08093C9050480F58134
:10548000E02D89EC95E00994089580E090E00E9479
:105490003C2480E090E00E94262410924A050E945D
:1054A0008715E9ECF5E086E0DF011D928A95E9F7C2
:1054B0001092C4051092C2051092C3050C9499294C
:1054C0008F929F92AF92BF92EF92FF920F931F9392
:1054D000CF93DF938090AB059090AC05A090AD0585
:1054E000B090AE0540914D0550914E0560914F052D
:1054F00070915005842A952AA62AB72ACFE1D0E0D8
:10550000E92EF12C082F10E0D501C4010C2E04C0A7
:10551000B695A795979587950A94D2F780FD04C014
:10552000219790F780E01AC0FE0184E0EE0FFF1F84
:105530008A95E1F7EE0DFF1D93E0EE0FFF1F9A95A0
:10554000E1F7E00FF11FEE0FFF1FE050FE4F8591D6
:1055500094910E946413019719F38C2FDF91CF91DE
:105560001F910F91FF90EF90BF90AF909F908F9001
:10557000089528E0929F800D1124682F6695669506
:105580006695982F977085E0689FB001112440E0E0
:1055900050E080E0FB01E40FF51FE053FA4F20815B
:1055A00030E0092E02C0369527950A94E2F7217063
:1055B0003327042E01C0220F0A94EAF7822B4F5F93
:1055C0005F4F4530510531F7089528E0929F800DD7
:1055D0001124E82FE695E695E695877051E001C025
:1055E000550F8A95EAF785E0E89FF0011124E05312
:1055F000FA4F20E030E070E04081CB01022E02C083
:10560000969587950A94E2F7817081958427852382
:10561000842781932F5F3F4F2530310569F7089527
:105620006093AB057093AC058093AD059093AE0588
:105630000C94452A0F931F9341E050E060E070E026
:1056400004C0440F551F661F771F8A95D2F74095F7
:105650005095609570958091AB059091AC05A091A7
:10566000AD05B091AE058A019B01082319232A23B9
:105670003B23C901B8011F910F910C94102B0F937C
:105680001F9341E050E060E070E004C0440F551FFC
:10569000661F771F8A95D2F78091AB059091AC0574
:1056A000A091AD05B091AE058A019B01082B192B85
:1056B0002A2B3B2BC901B8011F910F910C94102B81
:1056C00060E070E0CB010C94102B60934D0570935B
:1056D0004E0580934F05909350050C94452AFC018C
:1056E000808191810E94C31692959F70963079F0C7
:1056F00010F4925001C09A50923068F4803F69F0E3
:1057000018F4883E40F409C0843F29F406C0883E5E
:1057100020F0813F11F080E0089581E0089510921B
:105720004B0586E0E3E0F5E0DF011D928A95E9F79D
:105730000C94452A882321F00E9480150C9487152B
:105740000895882339F090914B05892B80934B0560
:105750000C94871508958823A9F19CEF980F913A2E
:1057600060F4E1E0F5E09281891301C01282319684
:1057700095E0E730F907B9F70DC090E2980F98303F
:1057800058F4877091E001C0990F8A95EAF7892F44
:105790000E9480150C9487159BE5980F933020F498
:1057A00080E090E00C943C2498E5980F973120F429
:1057B00080E090E00C9426248D3E20F00E944F283B
:1057C0000C9499290895CF93882309F49EC0C82F7B
:1057D0008CEF8C0F813A08F043C08091CF05813067
:1057E00081F030F08230A1F58C2FCF910C94BC2544
:1057F00080914B05823209F06AC08C2F0E940027ED
:105800002CC080914B058232C1F3C431C9F058F4E9
:10581000CB3069F0C031B9F482E08093CF0588E3E2
:105820000E94BC2552C0C93259F0C83361F483E5E7
:105830009DE00E94430880EE9FE00E94430845C01F
:105840001092CF0508C08EED9FE00E94430803C070
:105850001092CF053CC080E08170811156C037C0E6
:1058600080E28C0F883078F4C77081E090E001C04E
:10587000880FCA95EAF790914B05892B80934B05C9
:10588000CF910C948715EBE5EC0FE33040F4F0E09A
:10589000E95EFE4F808190E0CF910C943C24E8E5D6
:1058A000EC0FE73150F4F0E0EE0FFF1FE65EFE4F25
:1058B00080819181CF910C942624CD3E30F18C2FA4
:1058C0000E943E29CF910C94992981E0C5CFE3E055
:1058D000F5E089E095E02191C21721F08E179F072E
:1058E000D1F70DC0E1E0F5E08281C81301C012825A
:1058F000319685E0E730F807B9F70E9487156C2FDD
:1059000081E095E00E940C24BBCFCF9108951F93B6
:10591000CF93DF93CDB7DEB767970FB6F894DEBFAE
:105920000FBECDBF4B8B5C8B6D8B7E8B8F8B6111D4
:1059300010924A0586E09E01235F3F4FD901E82F70
:105940001D92EA95E9F795E0FE017396D901019061
:105950000D929A95E1F79C894E895F897B897D87B5
:105960009E876F87598B488BF901DE01179601904E
:105970000D928A95E1F7CE0107960E94E2168111F9
:105980003EC086E0FE013796DE01119601900D9231
:105990008A95E1F7FF81E8856A857B856115710548
:1059A00031F0EF3F31F481E0FF3F19F403C081E0B3
:1059B00001C080E080FD23C020910F0530E0C901C7
:1059C0000196877099274091400550E0841795070C
:1059D00079F1F983EA837D836C8396E0929FD0010D
:1059E000939FB00D1124A05FBA4FFE013196019034
:1059F0000D929A95E1F780930F050E944D1616E0DF
:105A00008091400590910F058917F9F0189FC0010A
:105A10001124805F9A4F0E94E2168823B1F0809192
:105A2000400590E001968770992780934005E8CF64
:105A30000E948F2B10920F0510924005E9E0F5E0CF
:105A400086E0DF011D928A95E9F767960FB6F89414
:105A5000DEBF0FBECDBFDF91CF911F9108951F9381
:105A6000CF93DF93182F117081FBDD27D0F982FBD4
:105A7000CC27C0F98091720580FF14C01F92CF938C
:105A80001F92DF931F921F9384EE9FE09F938F934B
:105A90000E94DC088DB79EB708960FB6F8949EBF9B
:105AA0000FBE8DBF8091AF05811105C0111102C0DD
:105AB0002D9A01C02D98D11102C02E9A01C02E98A6
:105AC000C11102C0589A01C05898DF91CF911F911F
:105AD00008958295982F937344E0949F9001112428
:105AE0008C7C86958695282B822F8575880F2A7A3F
:105AF0002695822B08950E948F2B2FEF84E39CE044
:105B0000215080409040E1F700C0000081E0809388
:105B1000E00080E28093D8001092C9008FE19EE4FB
:105B20000197F1F700C0000087E090EBDC01809363
:105B3000200690932106A0932206B09323069CE0B2
:105B400088E10FB6F894A895809360000FBE9093FB
:105B50006000FFCF8091AF058F5F8093AF050E94FB
:105B6000D72390935305809352050895CF93DF93E5
:105B70001EBC0E94D723EC010DB407FC0AC00E9492
:105B8000D7238C1B9D0B84369105B0F38EEF9FEFCE
:105B900002C08EB590E0DF91CF910895F999FECFC4
:105BA00092BD81BDF89A992780B50895A8E1B0E02B
:105BB00042E050E00C94022E262FF999FECF92BDC0
:105BC00081BDF89A019700B4021639F01FBA20BDC2
:105BD0000FB6F894FA9AF99A0FBE08950396272FF4
:105BE0000E94DD2D0E94DC2D252F0E94DD2D242F0B
:105BF0000C94DD2D0196272F0E94DD2D0C94DC2DB9
:105C0000DC01CB01FC01F999FECF06C0F2BDE1BD7C
:105C1000F89A319600B40D9241505040B8F708956B
:105C2000991B79E004C0991F961708F0961B881FEE
:105C30007A95C9F78095089597FB072E16F400947E
:105C400007D077FD09D00E94582E07FC05D03EF4FE
:105C5000909581959F4F0895709561957F4F089518
:105C6000EE0FFF1F0590F491E02D09940F9308307B
:105C700090F0982F872F762F652F542F432F322F98
:105C800022270850F4CF220F331F441F551F661FD1
:105C9000771F881F991F0A95B2F70F9108952A154B
:105CA0003B054C055D056E057F058007910708954E
:105CB000AA1BBB1B51E107C0AA1FBB1FA617B70732
:105CC00010F0A61BB70B881F991F5A95A9F780954E
:105CD0009095BC01CD010895FB01DC0104C08D91BC
:105CE0000190801921F441505040C8F7881B990B4E
:065CF0000895F894FFCFB7
:105CF600F904FF0101D921912272226E226A22D86B
:105D06002128081E0A1401818283E200E900EA00C4
:105D1600B500B600B700CD008301CC008A01920120
:105D260094012102230224022502260227022A02C6
:105D3600B300B4006F007000004000800020001027
:105D4600000800040001000240008000200010004E
:105D56000800040001000200407B22DC0661063FC9
:105D66000642075B07740791949734F7F6F5F43FFC
:105D76003F3F006D6B5F64656C6179006D6B5F69B9
:105D86006E74657276616C006D6B5F6D61785F73C2
:105D960070656564006D6B5F74696D655F746F5FD8
:105DA6006D6178006D6B5F776865656C5F6D6178B6
:105DB6005F7370656564006D6B5F776865656C5FC2
:0C5DC60074696D655F746F5F6D6178003B
:00000001FF
